:100000000C9484020C94BC020C94BC020C94BC02B0
:100010000C94BC020C94BC020C94BC020C94BC0268
:100020000C94BC020C94BC020C9441150C948314E7
:100030000C94B21A0C94BC020C94BC020C94BC023A
:100040000C94BC020C94BC020C94BC020C94BC0238
:100050000C94BC020C94741A0C94BC020C94BC0258
:100060000C94BC020C94BC020C94BC020C94BC0218
:100070000C94BC020C94BC020C94BC020C94BC0208
:100080000C94BC020C94BC020C94BC020C94BC02F8
:100090000C94BC020C94BC020C94BC020C94BC02E8
:1000A0000C94BC020C94BC020C94BC022508990868
:1000B0002D08F707FB073108FE0734083F08090839
:1000C0008F080D08430811084708710815084B08E8
:1000D0007B081B0851085B080208380805083B0824
:1000E00020085608670887088908F3072908A20826
:1000F000C208C808AA07BC08CE08D408DA08D00984
:10010000D009020A020A7C0B7C0B7C0B7C0B800A58
:10011000F40A050B050B9512BC126114BC12611494
:1001200004132713611416142A1418181B185718CF
:1001300067186E1879181719171917191719171939
:100140007C187F188418AA18CC18CF18D218F61863
:10015000000000000000000000000000000000009F
:10016000000000000000000000000000000000008F
:10017000000000007E0F00D4FFFFFFC700000078E2
:1001800000000000000000002A2B280000000000F2
:100190000000000000000000000000290000000036
:1001A0002C1E3420212224342627252E362D3738A4
:1001B000271E1F202122232425263333362E3738AD
:1001C0001F0405060708090A0B0C0D0E0F1011126B
:1001D000131415161718191A1B1C1D2F3130232D37
:1001E000350405060708090A0B0C0D0E0F10111235
:1001F000131415161718191A1B1C1D2F3130354CE6
:100200000660FF0961A1010962150026FF00952023
:10021000750881020963150026FF00952075089175
:1002200002C005010906A101050719E029E715002B
:100230002501950875018102950175088101050761
:10024000190029FF150026FF009506750881000595
:1002500008190129051500250195057501910295DB
:100260000175039101C009024200020100A0FA09D0
:1002700004000001030101000921110100012244D1
:1002800000070581030800010904010002030000C2
:10029000000921110100012222000705820320002C
:1002A00001070503032000011201000200000008FD
:1002B00017E161610100010200010C033600310009
:1002C0004B006500790000000A033000780043000D
:1002D0003700000004030904167C1E001F002000E4
:1002E00021002200230024002500260027002D00E5
:1002F0002E002A002B0014001A0008001500170019
:100300001C0018000C00120013002F0030003100F8
:10031000390004001600070009000A000B000D0058
:100320000E000F003300340000002800E1001D0023
:100330001B000600190005001100100036003700F0
:10034000380000000000E500E000E300E2000000EB
:1003500000002C0000000000E600215200006500B3
:100360000000E40029003A003B003C003D003E0054
:100370003F004000410042004300440045004C0063
:100380000100010052000100010001000100010014
:100390000100460047004800010001000100500034
:1003A00051004F000100010001000100010049005F
:1003B0004A004B00000001000100010001000100A3
:1003C00001000100010001004C004D004E00000042
:1003D0000000010001000100597C00000000010044
:1003E00000000000010001000000010000004C05B9
:1003F00001000100010001000100010001000100F5
:1004000001000100010001000100010001000100E4
:1004100001000100010001000100010001000100D4
:1004200001000100010001000100010001000100C4
:1004300001000100010001000100010001000100B4
:1004400000000100010001000100010001000100A5
:100450000100010001000100010000000000010096
:100460000100010001000000000001000000000088
:100470000100010000000100000001000100010076
:100480000100010001000100010001000100010064
:100490000100010001000100010001000100010054
:1004A0000100010001000100010001000100010044
:1004B0000100010001000100010001000100010034
:1004C0000100010001000100010001000000010025
:1004D0000100010001000100010001000100010014
:1004E0000100010001000000000001000100010006
:1004F00001000000000001000000000001000100F8
:10050000000001000000010011241FBECFEFDAE05F
:10051000DEBFCDBF04B603FE18C0809100029091EB
:100520000102A0910202B09103028730904BA740D4
:10053000B04B59F410920002109201021092020284
:1005400010920302E0E0F8E3099511E0A0E0B1E0C9
:10055000E2E7F1E402C005900D92A232B107D9F7AB
:1005600022E0A2E2B1E001C01D92A030B207E1F7A3
:100570000E945A160C94B7200C940000ABE0B0E037
:10058000E4ECF2E00C945120FC018481882311F406
:100590000C94B50B4F0121E0408151816281738140
:1005A00095810E94271F3C01815A9245D3014F97A4
:1005B00020F400EAA02702E5B027F401F581FA87CC
:1005C000FF2309F4C0C2AF3FB10571F068F0A9354F
:1005D000BC4719F01092440183C39091440181E01B
:1005E000892780934401BEC480914401882309F483
:1005F000E8C010924401A03CB10540F4A038B10518
:1006000008F073C0A034B105D0F505C0AF3FB10507
:1006100009F008F4A0C021E030E040E050E060E0E4
:1006200070E080E090E00A2F0E948820E091240191
:100630002E2BE09125013E2BE09126014E2BE091DF
:1006400027015E2BE09128016E2BE09129017E2B82
:10065000E0912A018E2BE0912B019E2B2093240107
:100660003093250140932601509327016093280180
:100670007093290180932A0190932B0132C321E0CA
:1006800030E040E050E060E070E080E090E08D011C
:10069000005411090E948820E0912C012E2BE0913A
:1006A0002D013E2BE0912E014E2BE0912F015E2B70
:1006B000E09130016E2BE09131017E2BE09132010F
:1006C0008E2BE09133019E2B20932C0130932D0132
:1006D00040932E0150932F016093300170933101AC
:1006E0008093320190933301FCC221E030E040E07E
:1006F00050E060E070E080E090E08D01005811096A
:100700000E948820E09134012E2BE09135013E2B90
:10071000E09136014E2BE09137015E2BE0913801DC
:100720006E2BE09139017E2BE0913A018E2BE09106
:100730003B019E2B209334013093350140933601C9
:1007400050933701609338017093390180933A01D7
:1007500090933B01C6C221E030E040E050E060E011
:1007600070E080E090E08D01005C11090E9488201B
:10077000E0913C012E2BE0913D013E2BE0913E01AA
:100780004E2BE0913F015E2BE09140016E2BE091FA
:1007900041017E2BE09142018E2BE09143019E2B83
:1007A00020933C0130933D0140933E0150933F0123
:1007B0006093400170934101809342019093430103
:1007C00090C2A034B105D0F450902401A09025012E
:1007D000B0902601E0902701F090280110912901A6
:1007E000F0912A01E0912B0121E030E040E050E05F
:1007F00060E070E080E090E00A2F5DC0A038B105B5
:10080000E8F450902C01A0902D01B0902E01E090C2
:100810002F01F090300110913101F0913201E091FF
:10082000330121E030E040E050E060E070E080E043
:1008300090E06D0100E4C01AD1083CC0A03CB105B5
:10084000E8F450903401A0903501B0903601E0906A
:100850003701F090380110913901F0913A01E0919F
:100860003B0121E030E040E050E060E070E080E0FB
:1008700090E06D0100E8C01AD1081CC050903C0106
:10088000A0903D01B0903E01E0903F01F09040010A
:1008900010914101F0914201E091430121E030E0EB
:1008A00040E050E060E070E080E090E06D0100EC3E
:1008B000C01AD1080C2D0E9488205222232E2A20F3
:1008C000342E3B20452E4E20F622E72EE1228F23A8
:1008D00089879E239B8721E030E040E050E060E084
:1008E00070E080E090E0A034B10580F08D01A03888
:1008F000B10518F4005411090AC0A03CB10518F460
:100900000058110904C0005C110901C00A2F0E949F
:10091000882059016A01F62FE72F8C01252D322DF1
:10092000432D542D6F2D7E2D89859B85EF2EFE2E18
:100930000E94A12009F0D4C1A03CB10548F4A03820
:10094000B10508F084C0A034B10508F042C005C06C
:10095000AF3FB10509F008F4B8C021E030E040E055
:1009600050E060E070E080E090E00A2F0E94882074
:10097000209530954095509560957095809590950F
:10098000E09124012E23E09125013E23E0912601F0
:100990004E23E09127015E23E09128016E23E09130
:1009A00029017E23E0912A018E23E0912B019E23D1
:1009B0002093240130932501409326015093270171
:1009C000609328017093290180932A0190932B0151
:1009D000C9C28D010054110921E030E040E050E02F
:1009E00060E070E080E090E00E94882020953095E3
:1009F000409550956095709580959095E0912C016B
:100A00002E23E0912D013E23E0912E014E23E09113
:100A10002F015E23E09130016E23E09131017E23AE
:100A2000E09132018E23E09133019E2320932C012B
:100A300030932D0140932E0150932F01609330018C
:100A40007093310180933201909333018BC28D01F9
:100A50000058110921E030E040E050E060E070E033
:100A600080E090E00E948820209530954095509538
:100A70006095709580959095E09134012E23E091DA
:100A800035013E23E09136014E23E09137015E238C
:100A9000E09138016E23E09139017E23E0913A0123
:100AA0008E23E0913B019E23209334013093350146
:100AB00040933601509337016093380170933901A8
:100AC00080933A0190933B014DC28D01005C110966
:100AD00021E030E040E050E060E070E080E090E055
:100AE0000E9488202095309540955095609570958E
:100AF00080959095E0913C012E23E0913D013E23AD
:100B0000E0913E014E23E0913F015E23E0914001E0
:100B10006E23E09141017E23E09142018E23E0911A
:100B200043019E2320933C0130933D0140933E01BD
:100B300050933F01609340017093410180934201C3
:100B4000909343010FC2AF3FB10511F008F0C4C04C
:100B5000A034B105D0F450902401A0902501B090AC
:100B60002601E0902701F090280110912901F091D1
:100B70002A01E0912B0121E030E040E050E060E00C
:100B800070E080E090E00A2F5DC0A038B105E8F485
:100B900050902C01A0902D01B0902E01E0902F01DB
:100BA000F090300110913101F0913201E091330168
:100BB00021E030E040E050E060E070E080E090E074
:100BC0006D0100E4C01AD1083CC0A03CB105E8F4B6
:100BD00050903401A0903501B0903601E09037017B
:100BE000F090380110913901F0913A01E0913B0108
:100BF00021E030E040E050E060E070E080E090E034
:100C00006D0100E8C01AD1081CC050903C01A090B2
:100C10003D01B0903E01E0903F01F0904001109105
:100C20004101F0914201E091430121E030E040E0D8
:100C300050E060E070E080E090E06D0100ECC01AF0
:100C4000D1080C2D0E9488205222A322B422252EE6
:100C50002E20362E3F20472E4122F8239E239987AF
:100C6000A034B105C0F08D01A038B10518F40054CE
:100C7000110908C0A03CB10518F40058110902C0C0
:100C8000005C110921E030E040E050E060E070E0FD
:100C900080E090E009C021E030E040E050E060E01A
:100CA00070E080E090E00A2F0E948820B22FA32FEE
:100CB0006A017B018C01E1E0252D3A2D4B2D522D4F
:100CC000632D742D8F2F9985AB2EBA2E0E94A120F3
:100CD00009F4E0E08E2F01C081E080FF43C154C1E0
:100CE000D301CD0197578038910508F055C10A2FDF
:100CF000A03108F037C18FEF93E00E94F21F8111FD
:100D000031C138E5C32E32E0D32E002379F0C1146F
:100D100024E0D20609F426C1C6010E94F21F811107
:100D200001C001503FEFC31AD30AEFCFCE010196A5
:100D30002C0188E0F20111928A95E9F72AE0322E1F
:100D400086010F5F1F4FC6010E94F21F89831A821E
:100D5000882309F407C1813009F041C07601F2E02F
:100D6000EF0EF11CC8010E94F21F8A83882309F448
:100D7000F9C09FEF980F933060F403E0C00ED11CD0
:100D8000C7010E94F21F8B83882309F4EBC01C82E9
:100D900029C0843031F55E0123E0A20EB11C02E0CF
:100DA00010E067013FEFC31AD30AC7010E94F21F88
:100DB000F50181935F01882309F4D4C08C3741F495
:100DC000E2E0F0E0EC0FFD1FE00FF11F10820AC01F
:100DD0000F5F1F4F76010730110519F7C3C0680177
:100DE00001C067018201F8012081222309F4A8CF04
:100DF000213009F053C08181813081F47801F2E023
:100E0000EF0EF11CF8018281893319F460E570E07E
:100E100002C060E070E00E940F1F15C0823049F4EC
:100E20007801F2E0EF0EF11CF80182810E946E1E43
:100E30000AC0833051F47801F2E0EF0EF11CF801A2
:100E400082810E942E1E870182C0843019F00F5FBC
:100E50001F4F7DC0F80122810E5F1F4F80E090E0A0
:100E600030E0205331092A30310568F4389EA00162
:100E7000399E500D1124C901840F951F0F5F1F4F1C
:100E8000F8012081EDCF009709F461C0EFE9FFE0A0
:100E90003197F1F700C000000197F5CFE22FF0E0A5
:100EA000E058FE4F2490822F86958695869590E097
:100EB000FC01E059FE4F64902770712C022E02C095
:100EC000759467940A94E2F7F1E06F227724FC01AD
:100ED000E05AFE4FA490B12C022E02C0B594A79404
:100EE0000A94E2F731E0A322BB24FC01E05BFE4F51
:100EF000E490F12C02C0F594E7942A95E2F781E0A2
:100F0000E822FF246114710419F081EE0E946E1E24
:100F1000A114B10419F086EE0E946E1E60E070E02C
:100F2000822D0E940F1FA114B10419F086EE0E94B9
:100F30002E1E6114710419F081EE0E942E1EE11420
:100F4000F10429F060E070E08CE20E940F1F0F5F57
:100F50001F4F49CF06E221EE41EE6AE17CE7C40172
:100F60000E944A1B80918801877009F4FEC3F40136
:100F70008581882309F4F9C38091BB0182FFF5C301
:100F800082E00E94760FF1C3F301E851FC47E7309D
:100F9000F10508F015C1ECC06D01E12CF12CFD014B
:100FA000E851FC47E730F10508F4E2C01092DD019A
:100FB000CD019057839708F015C184E090E00E941E
:100FC000FA1F9093BB018093BA01F601E150F047FC
:100FD000E232F10520F4EA5AFF4F0C94442080914C
:100FE000BA018160ACC08091BB018860B4C08091BF
:100FF000BA018260A4C08091BA0120C08091BA0178
:1010000088609DC08091BB011EC08091BB01826041
:10101000A2C08091BA01806192C08091BA018062C1
:101020008EC08091BA0180648AC00E940F1E809198
:10103000BA01806884C08091BA01886084607FC0F2
:101040008091BB018260816086C08091BA018E7FF1
:1010500076C08091BB01877F7EC08091BA018D7F71
:101060006EC08091BA0120C08091BA01877F67C0AD
:101070008091BB011EC08091BB018D7F6CC08091AF
:10108000BA018F7E5CC08091BA018F7D58C080917B
:10109000BA018F7B54C00E940F1E8091BA018F77D6
:1010A0004EC08091BA01877F8B7F49C08091BB0180
:1010B0008D7F8E7F50C08091BA0182FB222720F95C
:1010C00091E0922790FB82F990FB83F938C08091E0
:1010D000BB01982F909591708E7F892B90FB81F9A1
:1010E0003AC08091BA0186FB222720F991E092272D
:1010F00090FB86F924C00E940F1E8091BA0187FBE5
:10110000222720F991E0922790FB87F918C061E02F
:1011100001C060E08EE090E00E9410201EC080912F
:10112000BA0184FB222720F991E0922790FB84F9F1
:1011300006C08091BA01982F909590FB80F980931A
:10114000BA010BC08091BB0183FB222720F991E0FB
:10115000922790FB83F98093BB016091BA01709153
:10116000BB0184E090E00E942E200E940F1EFACE68
:10117000E858FF4F0C94442007E225EE45EE6BE162
:101180007CE7EDCE06E221EE40EE68E17CE7E7CEBB
:1011900007E225EE44EE69E17CE7E1CE06E221EECE
:1011A00042EE6CE17CE7DBCE07E225EE46EE6DE138
:1011B0007CE7D5CE08E221E045EE6EE17CE7CFCEBC
:1011C00006E160160CE7700609F0BEC28091450189
:1011D000811106C089E20E94DB1A0E943C0FC2CE38
:1011E00085E3F9CFA6312CE7B20781F48091930112
:1011F0008A7A91E009F490E090934501811104C04E
:1012000089E20E94E71AE9CF85E3FBCFA7373CE7E5
:10121000B30711F481E005C0A8378CE7B80749F49B
:1012200082E00E94DD1D43E062E081E00E948E11B9
:1012300099CE3D01C301805E92458097A8F4EA856E
:10124000E11116C0862D8F7101E010E002C0000F81
:10125000111F8A95E2F7602F83E090E00E94102032
:10126000802F0E94E91D7ECEFA85FF2309F443C03A
:10127000F3E06F16FCE77F0651F150F461142CE7A0
:101280007206B9F031E063163CE7730631F133C002
:101290008BE568168CE7780659F19CE569169CE7A2
:1012A0007906F1F0EAE56E16ECE77E0621F581E0BD
:1012B00020C00E940F1EFFEF04E32CE0F15000401D
:1012C0002040E1F700C000000E94501A4BCE6FEFA3
:1012D0007FEF80E090E00E942E200E94DC1F42CE33
:1012E0008091BB0182FB882780F991E0892701C0AA
:1012F00080E00E948D0FF401858100811181882397
:1013000049F0C8010E94281DF82E682FC8010E94CC
:10131000981D04C0C8010E94641DF82EB8018F2DCD
:101320000E949E0D0E94AC0D8C01C82EF401F58028
:10133000E680E2949FE0E92280918801877001F1C4
:10134000FF20F1F0812F807F803469F080E2800FF0
:101350008830B0F0812F807E803229F4F1E0F017E0
:1013600078F4EE2069F08091BB0182FF09C082E031
:101370000E94760F809188018770DD24D3948111BB
:10138000D12CB12EB2948FE0B8228B2D90E08C300E
:10139000910508F0B1C1FC01E158FF4F0C944420C5
:1013A000812F807F1F70882311F01295107FFF20FE
:1013B000B9F0112309F48EC180E2800F883010F05B
:1013C000C11006C080919301182B1093930105C0A2
:1013D00080918A01182B10938A010E943C0F7AC1D8
:1013E000802F0E942E1E112309F486C1005E083052
:1013F00080F1CC2071F1109580918A01182310930F
:101400008A012AC0812F807F1F70803211F01295CF
:10141000107FCC2029F021E0C21609F44CC057C03F
:101420008091BB0182FD1BC0FF2069F0112339F0C0
:1014300080919301182B109393010E943C0F80E040
:101440000E946E1E59C180E00E942E1E112309F4D5
:1014500053C1812F0E94350F0E943C0F4DC1FF20C8
:1014600081F0EE20C1F131E0E31246C180918901A3
:10147000912F9823191709F43FC1182B1093890154
:101480003BC1E11039C1812F0E941D1E809189014D
:10149000912F982329F0912F90958923809389018A
:1014A00090914601812F892309F426C1109591233B
:1014B0009093460121C1FF2029F085E08E1508F4A4
:1014C0001BC109C094E09E1508F416C115C0FF2089
:1014D00031F0E110FFC0812F0E94241E0DC1EE20CB
:1014E00059F0093309F005C1EFEFF7EE23E0E150C1
:1014F000F0402040E1F7FBC0812F0E941D1EFCC080
:10150000812F8370A9F5F110FBC0402F42954695BD
:101510004770440F440F802F8F7090E09C01042E81
:1015200001C0220F0A94EAF704FF08C08FE090E0A0
:1015300001C0880F4A95EAF7809501C080E01695B2
:1015400016951370123069F088F49091940111305F
:1015500019F0822B892302C0922B892B0E94E91D4E
:10156000CFC0822B909194018927F8CF822BF6CFA0
:10157000FF2019F0812F817001C08695882309F41E
:10158000BFC0402F429546954770440F440F802FAF
:101590008F7090E09C01042E01C0220F0A94EAF79C
:1015A00004FF08C08FE090E001C0880F4A95EAF779
:1015B000809501C080E0169516951370123059F091
:1015C00078F49091B901113019F0822B892309C068
:1015D000922B892B06C0822B9091B901892701C0DB
:1015E000822B0E94CD1D8CC01F70FF2039F0812FEF
:1015F0000E94DD1D802F0E94241E82C0802F0E9429
:101600001D1E812F0E94D01D7BC0802F32EFC3167C
:1016100081F13C1538F090EFC91659F0E1EFCE1684
:1016200019F154C0F3EFCF1659F124EFC216C1F0EF
:101630004DC0FF2081F034E03E1508F45DC01F71FD
:1016400081E090E0012E01C0880F0A94EAF79091A2
:10165000B901892720C085E08E1508F44DC0EFCF71
:101660008091BB0182FD1AC0FF2029F0812F8F716C
:1016700020C0FF20D9F3812F8F710E94D01D3CC064
:10168000FF2041F01F7181E0012E01C0880F0A94F4
:10169000EAF701C080E00E94CD1D2EC0FF2061F05E
:1016A000812F8F7198E0899F9001112423602093EE
:1016B00088010E94DD1D20C081E00E94760FE1E0DC
:1016C000EE15D0F482E00E94760F16C0FF2021F0C4
:1016D000EE2061F2802FB4CEEE2069F2893349F416
:1016E000FFEF27EE33E0F15020403040E1F700C03B
:1016F0000000802F0E942E1E88EF8B0D843010F486
:101700000E94001BDD20A9F08091880180FD11C09E
:10171000F40115828695869586950E94DD1DC4018B
:101720000E94BE02809188018695869586950E94CA
:10173000D01D20E0F4014081518162817381848158
:1017400095810E94271F11C097E769169CE77906CB
:1017500011F481E007C0E8E76E16ECE77E0609F0B9
:1017600069CD82E00E94D01D5ECD2B96E2E10C9403
:101770006D2080E008959091BA0192FF10C041E081
:10178000282F2471243009F040E031E0282F2871FF
:10179000283009F030E0431711F02CE0822793FF46
:1017A00010C041E0282F2471243109F040E031E0DD
:1017B000282F2871283109F030E0431711F02CE070
:1017C00082273091BB0130FF10C051E0282F2171DA
:1017D000213009F050E041E0282F2871283009F02D
:1017E00040E0541711F029E0822731FF10C041E09A
:1017F000282F2171213109F040E031E0282F287194
:10180000283109F030E0431711F029E0822794FDD8
:10181000877E08958238910569F1B0F4813391058E
:1018200009F475C048F48932910509F467C08A3219
:10183000910509F471C008958533910509F459C0E3
:1018400089339105B9F00895833E910589F138F403
:10185000803E9105D1F0823E910529F10895863EA2
:101860009105C9F1873E9105D9F1843E910509F0B2
:101870006CC027C02091BA0120FD57C021FD55C082
:101880002091BB0123FD5BC008958091BA0180FDCA
:1018900048C08091BB0180FF48C08091BA0184FD9F
:1018A00046C083EE51C08091BA0182FF3CC0F5CFA3
:1018B0008091BA0182FD37C08091BB0180FD35C0A7
:1018C000ECCF8091BB0181FF36C08091BA0184FDCD
:1018D0002EC087EE39C08091BA0183FF2AC0F5CFB0
:1018E0008091BA0183FD25C08091BB0181FD23C099
:1018F000ECCF8091BA0185FD22C01FC08091BA0152
:1019000085FD1BC08091BB0183FF19C00AC0809177
:10191000BA0186FD16C017C08091BA0186FD13C0BA
:1019200010C089E311C082EE0FC080EE0DC080E0D0
:101930000BC086EE09C084EE07C085E305C089E2CE
:1019400003C08AE201C081E390E0089520918701FD
:1019500090914E0157E02917A9F030E0529FF00115
:10196000539FF00D1124E15BFE4F7181761306C089
:101970007081781303C07581741306C02F5F3F4FC9
:101980002770E9CF80E0089581E00895F894E82F6A
:10199000E295EF70F0E031A1282F2F7081E090E008
:1019A00001C0880F2A95EAF7982F9095932391A369
:1019B00092A1892B82A378940895AAE0B0E0E3EE87
:1019C000FCE00C945320AE014F5F5F4F7A018AE038
:1019D000FA0111928A95E9F70EE011E06A0193E1AC
:1019E000492E91E0592E66246394712C31E2832EA6
:1019F00031E0932EF80180818F3F09F446C0F894BE
:101A0000E82FE295EF70F0E021A18F70A30102C0F2
:101A1000440F551F8A95E2F7CA01922F982B91A384
:101A200092A18095892382A3789400C0E3E1F1E03C
:101A300021E030E0A12CB12C41914F3F89F0A42F3F
:101A4000A295AF70B0E090968C9190E04F7002C07C
:101A5000959587954A95E2F780FD02C0C90102C0BD
:101A600080E090E0A82AB92A220F331F8E169F0625
:101A700019F7F80180818F3F11F00E94C60CF0EA3F
:101A8000FA95F1F7F601B182A0820F5F1F4FF2E0E5
:101A9000CF0ED11C4016510609F0ACCF4AE050E001
:101AA000B7018FEA91E00E94AA20892B91F08AE089
:101AB000F701AFEAB1E001900D928A95E1F781E07C
:101AC000809399010E94A61A9093980180939701A0
:101AD00017C080919901882399F020919701309146
:101AE00098014FB7F8948091E1019091E201A091A3
:101AF000E301B091E4014FBF821B930B059710F4F3
:101B000080E018C04AE050E06FEA71E087EC91E0B5
:101B10000E94AA20892B59F08AE0EFEAF1E0A7ECB5
:101B2000B1E001900D928A95E1F781E001C080E07B
:101B3000109299012A96E0E10C946F20753048F4D8
:101B40006E3038F4843028F4462F672F0E94561CDC
:101B5000089580E090E008951F93CF93DF930E9453
:101B60000A0CEC01C11582E5D807C8F5C11590E54E
:101B7000D90708F0BBC0C83ED105C0F4C03ED105AE
:101B800008F0DDC0C53AD10550F4C430D10508F0E5
:101B9000D6C0219709F0D0C081E090E0D1C0CD3C03
:101BA000D10508F4C9C0CE019065CAC0C11580E452
:101BB000D80708F05AC0C11590E2D90708F0AFC0A5
:101BC000C11581E0D80708F4B7C08D2F0E94BB0B68
:101BD000182FCE0199270E940A0C1F71ABC0C03884
:101BE00092E5D90720F5C03682E5D80708F061C034
:101BF000C03492E5D90708F04AC0C03282E5D80760
:101C0000F0F54C2F4695469590E2499FA00111248E
:101C1000C37021E030E0C90102C0880F991FCA9546
:101C2000E2F7EA01C82BD92BCE019D6889C0C03CE0
:101C300092E5D90768F48C2F8F71C03AD24508F02D
:101C40004CC090E0D82FCC27CE01846F906A78C02A
:101C5000C03E82E5D80708F06FC0CF71DD27DC2FCA
:101C6000CC27CE01806F906A6BC0CE0199270E946D
:101C70000A0CCC27DF70D06A8C2B9D2B61C0CF71F2
:101C8000D0E0DC2FCC27CE01816F906A59C08C2F19
:101C90008F718695869590E2899F90011124C3707B
:101CA00081E090E002C0880F991FCA95E2F79C6816
:101CB00011C08C2F8F718695869590E2899F900137
:101CC0001124C37081E090E002C0880F991FCA956B
:101CD000E2F79A68822B932B33C00E94BB0B8F7163
:101CE00090E0D82FCC27CE0190622AC08C2F8F7124
:101CF0000E94BB0B95E0D695C7959A95E1F7CF70FA
:101D0000D0E0DC2FCC27282F30E084FF05C084E012
:101D1000220F331F8A95E1F7D069CE01DBCF8D2FDB
:101D20008F710E94BB0B182FCE0199270E940A0CBD
:101D30001F719062912B04C080E090E001C0CE0141
:101D4000DF91CF911F910895A6E0B0E0EAEAFEE0AE
:101D50000C945F200E94A61A8C01809195019091AD
:101D600096010817190781F019821A820E94A61A93
:101D7000682F49815A81792F80E090E00E944C1FA2
:101D800010939601009395012696E4E00C947B2035
:101D9000A8E0B0E0EEECFEE00C94612065EE7EEF92
:101DA00080E090E00E942E2060E082E090E00E94BF
:101DB000102081E08093940161E083E090E00E9434
:101DC000102060E074E184E090E00E942E2060E04A
:101DD00086E090E00E94102060E087E090E00E94A2
:101DE000102040E050E0BA0188E090E00E942220FC
:101DF00060E083E290E00E94102060E08CE090E0E0
:101E00000E94102060E08DE090E00E941020198276
:101E10001A821B821C821D821E821F82188648E045
:101E200050E067E170E0CE0101960E94002040E0A2
:101E300050E0BA018FE190E00E94222080E00E94F1
:101E4000121B0E94461C40E050E0BA018FE090E077
:101E50000E94222040E050E0BA0183E190E00E941D
:101E600022202896E2E00C947D20809590919301A9
:101E700089238093930108959091930180918A0121
:101E8000892B90918901992379F0892BE3EDF1E079
:101E900027E090E0215029F031913323D9F39F5F5F
:101EA000F9CF9111109289018093D10148E050E05F
:101EB0006BE871E081ED91E00E94AA20892BA9F0E6
:101EC00088E0E1EDF1E0ABE8B1E001900D928A9598
:101ED000E1F7E091DE01F091DF01309731F002800F
:101EE000F381E02D81ED91E00995089590918801AD
:101EF0008095892380938801282F277069F498178B
:101F000059F09091BB0192FF07C086958695869502
:101F10000E94D01D1092880108959091BB0192FB00
:101F2000222720F9281779F080FB92F99093BB01C2
:101F30006091BA017091BB0184E090E00E942E2074
:101F400082E00E94760F08958091870190914E0162
:101F5000891719F08F5F8770FBCF0895CF93DF93B8
:101F600080914D0182958F7009F04EC080914C0197
:101F7000882309F449C08091870140914E01509116
:101F8000480160914701C0914901D0914A0177E031
:101F90008417D1F190E0789FF001799FF00D112422
:101FA000DF01A15BBE4F14962C911497222349F1B7
:101FB00011962C911197251324C02C91261321C022
:101FC00015962C91159721111CC012962D913C91BC
:101FD00013972C1B3D0B283C310598F480914D0143
:101FE0008F70806180934D01EB5AFE4F80818F701E
:101FF0008061808387E491E00E94BE020E94A40F6A
:1020000003C001968770C4CFDF91CF910895A4E1FA
:10201000B0E0EDE0F0E10C9457208C0186E0F8018F
:10202000DE011F9601900D928A95E1F7F8018481F7
:10203000E58097E4892E91E0992E90914B019111C2
:1020400020C0882309F463C1EE2009F442C0C8010E
:102050000E94EC1DF82E8823E1F187E0F801D401FD
:1020600001900D928A95E1F780914B01813031F416
:1020700080914701909148010E94571D0E94AE0F28
:1020800048C1F801D080C180A280B380F0904C019B
:102090002091490130914A01FF2009F4E7C0A501D0
:1020A000421B530B483C510508F09DC0882309F49E
:1020B00030C180914D01282F207F9091480122232B
:1020C00061F09C1509F460C0C8010E94EC1D8111EB
:1020D00063C0C8010E94BE021AC19C1113C0909136
:1020E00047019D110FC0E1100DC08F70806180937A
:1020F0004D0187E491E00E94BE0280914D01F801FC
:10210000868303C1E1103AC040E06C2D8D2D0E9402
:10211000A60C40E06C2D8D2D0E94A60CE82E81119E
:10212000F4C0DF86C88A8F8598890E94571D292FA1
:1021300022952F70243020F49F70223028F009C09F
:102140002A50223080F014C0992349F0811107C031
:1021500013C0992321F0F8019681907F69F0805E89
:10216000883030F409C0803F38F0815F833020F040
:10217000C8010E94BE02EF2CFE2CCBC080914D0105
:10218000816080934D01C1C0909147019D119CCF0A
:10219000E1109ACFF80198C0EE2009F49ACF20916F
:1021A0004D01822F82958F7090E002978CF0809184
:1021B00047019091480199878887BB86AA868091BC
:1021C0004B018C871D862E87CE0108960E94BE0289
:1021D00087E0F801A7E4B1E001900D928A95E1F75C
:1021E0000E94AE0F94C090914D01292F207F51F491
:1021F00087E491E00E94BE0287E0F40111928A9583
:10220000E9F783C0882309F484C0809148018C11C8
:102210000CC0809147018D1108C0E11006C0F80183
:102220009683C8010E94BE026AC0C8010E94EC1DCC
:10223000882309F44ECFEE2009F44BCF20914D01B5
:10224000822F82958F7090E0029714F2809147015F
:10225000909148019A838983BC82AB8280914B0123
:102260008D831E822F83CE010196B0CFA21AB30AAE
:10227000F8ECAF16B10408F042C0882309F447C057
:10228000FE2CEE2009F425CF809148018C1129C045
:10229000809147018D1125C090914D0190FD18C08E
:1022A000892F82958F70282F30E02115310581F01C
:1022B000F80196832F30310541F08F5F982F92956A
:1022C000907F86818F70892B8683C8010E94BE0211
:1022D00087E0F801A7E4B1E001900D928A95E1F75B
:1022E00018C0C8010E94EC1D811172CF80914D0170
:1022F000816080934D01C8010E94BE020AC087E040
:10230000F40111928A95E9F704C0F12C02C0FF2470
:10231000F3948F2D6496ECE00C9473209091B901A6
:1023200021E030E0F90101C0EE0F8A95EAF7D9010A
:1023300002C0AA0FBB1F6A95E2F7BD016E2B01C058
:10234000220F4A95EAF7892F8623681303C0892F45
:10235000822B03C02095822F89230E94CD1D0895D2
:10236000AAE2B0E0E6EBF1E10C946020E7EAF1E0EC
:102370008091F100819321E0EF3AF207C9F7809153
:10238000A801833009F461C030F4813071F08230EB
:1023900009F4A0C0B7C08A3009F48CC08B3009F4AE
:1023A0006CC0893009F0AEC020C08091A701813A8D
:1023B00009F0A8C08091E800877F8093E8008091B1
:1023C000AB019091AC01892B21F468E08BE991E09D
:1023D00003C060E080E090E070E00E94A01980916E
:1023E000E8008B778093E8008DC08091A70181324F
:1023F00009F088C08091AB019091AC01892B09F064
:1024000081C08091E800877F8093E8008091E80098
:1024100082FD05C08091A5018111F8CF73C0209184
:10242000F3008091F20090E0922B029731F48091BA
:10243000F100813011F0863021F48091F100809319
:1024400001018091E8008B7759C08091A701813A02
:1024500009F058C08091AB019091AC01892B09F033
:1024600051C08091E800877F8093E8008091E80068
:1024700080FFFCCF809102013CC08091A701813296
:1024800009F040C08091AB019091AC01892BD1F54E
:102490008091E800877F8093E8000E944C1981E0DA
:1024A0009091A901911101C080E0809302010E94E6
:1024B0000F1E28C08091A701813221F58091E8008C
:1024C000877F8093E8000E944C198091AA01809335
:1024D000000118C08091A701813AA1F48091E80021
:1024E000877F8093E8008091E80080FFFCCF809197
:1024F00000018093F1008091E8008E778093E800DE
:102500000E944C198091E80083FFDBC18091A701F4
:102510009091A801492F50E04A30510508F0D1C1EF
:10252000FA01E557FF4F0C944420803821F082389F
:1025300009F0C7C108C08091A3019091A40199231B
:1025400089F082600FC08091AB018F70873008F0F6
:10255000B8C18093E9008091EB0085FB882780F962
:102560001092E9009091E800977F9093E8008093A3
:10257000F1001092F10066C1282F2D7F09F0A1C152
:10258000882319F0823061F09CC18091A9018130CB
:1025900009F097C1933009F080E08093A4012EC028
:1025A0008091A90181112AC08091AB018F702FEF1A
:1025B000280F263008F085C18093E9002091EB00B8
:1025C00020FF1CC0933021F48091EB00806214C086
:1025D0009091EB0090619093EB0021E030E0A90135
:1025E00002C0440F551F8A95E2F74093EA0010920B
:1025F000EA008091EB0088608093EB001092E90084
:102600008091E800877F21C181115BC11091A901F0
:102610001F778091E3008078812B8093E300809185
:10262000E800877F8093E8000E944C198091E800C1
:1026300080FFFCCF8091E30080688093E30011115C
:1026400002C082E001C083E08093A5013AC18058B6
:10265000823008F036C18091A9019091AA018C3D89
:1026600053E0950779F583E08A838AE289834FB73F
:10267000F894DE01139620E03EE051E2E32FF0E013
:1026800050935700E49120FF03C0E295EF703F5F45
:10269000EF708E2F90E0EA3010F0C79601C0C09620
:1026A0008D939D932F5F243149F74FBF8091E800B0
:1026B000877F8093E8006AE270E0CE0101960E9475
:1026C000A019AEC04091AB015091AC01292F332726
:1026D00023303105A9F068F42130310509F400C137
:1026E0002230310509F0EDC082E490E0E6E6F2E048
:1026F00044C02132310521F12232310571F1E1C0AE
:10270000992781309105A1F058F0029709F0D9C0BE
:10271000EAEBF2E0E4918E2F90E0EAEBF2E02AC0DF
:10272000E4EDF2E0E4918E2F90E0E4EDF2E022C0DF
:10273000E8ECF2E0E4918E2F90E0E8ECF2E01AC0D1
:102740004115510509F4D1C04130510509F0B9C016
:1027500089E090E0E1E9F2E010C04115510509F48B
:10276000C9C04130510509F0ACC082E290E0E0E020
:10277000F2E003C0009709F4A4C02091E800277F8D
:102780002093E8002091AD013091AE0182179307AC
:1027900008F49C0140E02115310589F18091A501E3
:1027A000882309F43DC08530D9F18091E80083FD8C
:1027B00037C08091E80082FD2FC08091E80080FF43
:1027C000EACF4091F3008091F20090E0942B211524
:1027D000310559F08830910540F444914093F1005F
:1027E0003196215031090196F2CF41E0089709F066
:1027F00040E08091E8008E778093E800CCCF4111D3
:10280000CDCF0AC08091A501882351F0853041F0D9
:102810008091E80083FD04C08091E80082FFF2CF40
:102820008091E8008B778093E8004BC0803809F0F6
:1028300048C08091E800877F8093E8008091A601DE
:102840008093F1008091E8008E778093E8000E94E9
:102850004C1937C0811135C08091A9019091AA010E
:102860009927029774F58091E800877F8093E800AC
:102870001091A9011093A6010E944C19111106C0D4
:102880008091E30087FD02C081E001C084E0809375
:10289000A50142E061EC81E00E946B1942E261EC2B
:1028A00082E00E946B1942E260EC83E00E946B19A7
:1028B0008091A501843011F081E001C082E0809315
:1028C00003018091E80083FF1AC08091E800877FB0
:1028D0008093E8008091EB0080628093EB000FC052
:1028E00082E190E0E8EAF2E048CF89E090E0E8E7B2
:1028F000F2E043CF84E490E0E2E2F2E03ECFAA9639
:10290000E3E00C947C201F920F920FB60F921124DB
:102910002F933F934F935F936F937F938F939F93E7
:10292000AF93BF93CF93DF93EF93FF93C091E900F1
:10293000CF708091EC00D82FD17080FDD0E810923C
:10294000E9008091F000877F8093F00078940E94E6
:10295000B0111092E9008091F00088608093F0003F
:10296000CD2BCF70C093E900FF91EF91DF91CF9114
:10297000BF91AF919F918F917F916F915F914F9197
:102980003F912F910F900FBE0F901F901895E8ED7B
:10299000F0E080818E7F80831092E2001092DA0056
:1029A0001092E100A0EEB0E08C9181608C93808168
:1029B0008F77808319BCA7EDB0E08C918E7F8C93CC
:1029C00080818F7E808310929A010895A0E0B0E00C
:1029D000ECEEF4E10C945B20C8EDD0E088818F7EB2
:1029E0008883E7EDF0E080818160808384E082BFAE
:1029F00081E080939A0188818E7F888302EE10E0C7
:102A0000F80110821092DA0081EEC82ED12CF60166
:102A1000108288818F778883888180688883888105
:102A20008F7D888319BC1092A5011092A601109287
:102A3000A4011092A30190EEE92EF12CF701808100
:102A40008B7F808388818160888342E060E080E0C2
:102A50000E946B19F60180818E7F8083F80180814E
:102A600081608083808188608083F70180818E7F90
:102A70008083888180618883CDB7DEB7E8E00C94DD
:102A800077201F920F920FB60F9211242F933F932E
:102A90004F935F936F937F938F939F93AF93BF9366
:102AA000EF93FF938091E10082FF09C08091E200E3
:102AB00082FF05C08091E1008B7F8093E1008091CF
:102AC000DA0080FF2AC08091D80080FF26C0809164
:102AD000DA008E7F8093DA008091D90080FF18C0E1
:102AE00080E189BD82E189BD09B400FEFDCF81E0AE
:102AF0008093A50180919A0181110FC00E94C71493
:102B00000E94E6148091E20084608093E20005C098
:102B100019BC1092A50110929A018091E10080FFEA
:102B20001AC08091E20080FF16C08091E2008E7F83
:102B30008093E2008091E20080618093E2008091C6
:102B4000D80080628093D80019BC85E08093A501ED
:102B500083E0809303018091E10084FF37C080917E
:102B6000E20084FF33C080E189BD82E189BD09B400
:102B700000FEFDCF8091D8008F7D8093D80080919A
:102B8000E1008F7E8093E1008091E2008F7E809350
:102B9000E2008091E20081608093E2008091A601D2
:102BA000882311F084E007C08091E30087FD02C014
:102BB00081E001C083E08093A5018091A50184306C
:102BC00011F081E001C082E0809303018091E10077
:102BD00083FF2CC08091E20083FF28C08091E10038
:102BE000877F8093E10082E08093A5011092A60187
:102BF0008091E1008E7F8093E1008091E2008E7FE2
:102C00008093E2008091E20080618093E20042E0E4
:102C100060E080E00E946B198091F00088608093F2
:102C2000F00081E08093030180930201FF91EF9116
:102C3000BF91AF919F918F917F916F915F914F91D4
:102C40003F912F910F900FBE0F901F9018952091DC
:102C5000E4003091E50095E64091EC00842F81700E
:102C600040FF23C08091E80080FD1DC08091A50138
:102C7000882399F0853099F08091EB0085FD11C093
:102C80004091E4005091E5002417350729F3915055
:102C900011F09A01E1CF84E0089582E0089583E085
:102CA000089581E0089580E008954091E80042FF92
:102CB000DDCF0895A6E2B0E0E0E6F6E10C94512005
:102CC00085B7806885BF85B7806885BF84B7877FF3
:102CD00084BF0FB6F894A8958091600088618093B6
:102CE0006000109260000FBE90E080E80FB6F8948C
:102CF00080936100909361000FBE81E08093030197
:102D000089EB9BE090932301809322010E94C714DA
:102D10000E94E6148091E20084608093E20078943F
:102D20008091A5018823A1F01091E9001F70909176
:102D3000EC00892F817090FD80E8182B1092E9003B
:102D40008091E80083FD0E94B0111F701093E9008C
:102D500082E084BD93E095BD9AEF97BD80936E00AD
:102D60000E94311B811102C00E94461C0EE011E03E
:102D7000D8018D918D018F3F11F00E94C60CB1E0FA
:102D800003311B07A9F703E111E0F80181918F01DD
:102D90008F3F11F00E94C60CF1E001321F07A9F726
:102DA0008AE0E7ECF1E0DF01282F1D922A95E9F790
:102DB000EFEAF1E0DF011D928A95E9F780E090E00B
:102DC0000E94FA1F853E9E4F21F40E94311B811103
:102DD00002C00E94C80E82E090E00E94F21F809321
:102DE000DA0184E090E00E94FA1F9093BB01809387
:102DF000BA010E94DD0CEFEFF6E721E0E150F04070
:102E00002040E1F700C000000E94DD0C8091C70166
:102E100080FF08C06FEF7FEF80E090E00E942E20DF
:102E20000E94501A83E090E00E94F21F0E94E91D68
:102E300084E091E09093DF018093DE01A1ED4A2EC2
:102E4000A1E05A2E8E010F5F1F4F8091A5018530A2
:102E500009F03EC08091A501853009F035C0809110
:102E6000A501843021F11092E00188E190E0A0E416
:102E70000FB6F894A895809360000FBEA0936000F1
:102E800083B7817F846083BF83B7816083BF789479
:102E9000889583B78E7F83BF0FB6F894A8958091ED
:102EA0006000886180936000109260000FBE0E94F5
:102EB000DD0CE7ECF1E081919191892B09F0C0C123
:102EC0004E165F06C1F7C6CF0E940F1E0E94001B60
:102ED0000E94DD0CECEBEE2EE1E0FE2EF7EC6F2E07
:102EE000F1E07F2ED301F701219131918D919D91D8
:102EF0008227932721E0E63CF20719F0892BA1F302
:102F000005C0892B19F40E94A40E3FC0312CD301B7
:102F10008D909D903D01F701A080B180A824B92437
:102F2000A114B10449F1212CCC24C394D12CC501A6
:102F30008C219D21892BB9F029A23AA20E94A61AC0
:102F40009CA38BA3F1E0FDA391E094012C213D21F2
:102F5000232B09F490E09EA349A15AA16BA17CA167
:102F60008DA10E944C1F2394CC0CDD1C2EE022125C
:102F7000DECFD7018D929C923394B2E0EB0EF11C20
:102F8000E5E03E12C4CF0E949A1A0E94001B909165
:102F9000C601891721F08093C6010E949A1A809178
:102FA000A501843009F051CF83E08093E90080913E
:102FB000E80082FF4ACF8091E80085FF23C00E948D
:102FC000271681111DC050E2C52ED12CCE010196CD
:102FD0007C0109C08091F100D7018D937D01B1E0A2
:102FE000CB1AD10869F08091E80085FDF3CF80917C
:102FF000E8008B778093E8000E942716882399F3D6
:1030000091E001C090E08091E8008B778093E80028
:10301000992309F41ACFE9818E2F90E0FC013197B2
:10302000E331F10508F003C1EB56FF4F0C94442047
:103030001A828CE067C08A81823009F41EC150F484
:10304000813009F0F4C00E949A1A9B838C837D839F
:103050006E83EFC0833041F0843009F0E8C01B82FA
:103060001C821D821E82E5C06B81DE01119680E00C
:1030700090E0262F30E0A901480F591F4530510537
:1030800008F0D7C0E62FE80FF0E0EE0FFF1FE9537E
:10309000FE4F4081518113965C93139714964C9385
:1030A0001497019612968E30910529F7C2C08A8135
:1030B000823021F0853009F4BCC0B9C06B817C81BD
:1030C0008D819E810E944A200E940D1BB2C04C81BE
:1030D0006B818A810E94561C9D83D6C02D813E81C2
:1030E0003227232732274C816B818A810E94EA1B79
:1030F000A0C00E94111C9DC0E0E1EA839AC0F1E0EB
:10310000FA8388EA8B8395C0EA80FB80FE24EF2453
:10311000FE24AC80B12C6801C701885A9D4F9601EE
:10312000201B310B2A153B0508F083C028EAE21664
:1031300021E0F20630F40E94F21FD60114968C931F
:1031400002C0F6011482FFEFEF1AFF0A2FEFC21A36
:10315000D20AE2CFEA80FB80FE24EF24FE24AC807A
:10316000B12C6801C701885A9D4F9601201B310B75
:103170002A153B0508F05DC0A8EAEA16A1E0FA06A8
:1031800020F4F60164810E941020FFEFEF1AFF0A7D
:103190002FEFC21AD20AE6CF0E94DA1B4AC084E09F
:1031A0008A8347C0EA80FB80FE24EF24FE24AC80A3
:1031B000B12C6801C70188969601201B310B2A1596
:1031C0003B05B8F5A0E3EA16A2E0FA0628F40E944F
:1031D000F21FF601848303C0D60114961C92BFEF40
:1031E000EB1AFB0AEFEFCE1ADE0AE4CFEA80FB808F
:1031F000FE24EF24FE24AC80B12C6801C701889620
:103200009601201B310B2A153B0598F4F0E3EF16CD
:10321000F2E0FF0628F4D60114966C910E9410206B
:10322000BFEFEB1AFB0AEFEFCE1ADE0AE7CF8FEF04
:10323000898340E250E0B80182E00E94FE1905CE89
:103240008091A401882309F405CEB0E1B9BDE2E183
:10325000E9BD09B400FEFDCF8091D8008F7D809339
:10326000D8008091E00082608093E0008091E000CF
:1032700081FDFCCF0E940F1EEDCD87E290E00E9401
:10328000F21F1B821C821D828E83D3CF0895089566
:1032900008958091010108958091A70187FF11C0D1
:1032A0008091E80082FD05C08091A5018111F8CFD1
:1032B00011C08091E8008B770BC08091A501882315
:1032C00049F08091E80080FFF8CF8091E8008E7788
:1032D0008093E8000895982F973068F59093E9005F
:1032E000981739F07091EC002091ED005091F000AA
:1032F00003C0242F762F50E021FD02C09F5FECCF4A
:103300003091EB003E7F3093EB003091ED003D7F3C
:103310003093ED003091EB0031603093EB0070930F
:10332000EC002093ED005093F0002091EE0027FD7B
:10333000E5CF80E008958F708093E90081E00895E3
:103340002091AD013091AE012617370748F0611585
:10335000710539F42091E8002E772093E80001C030
:10336000B901FC0120E06115710579F18091A50199
:103370008823F1F18530F1F18091E80083FD3CC0B4
:103380008091E80082FD2EC08091E80080FFEBCFA5
:103390002091F3008091F20090E0922B611571056D
:1033A00051F08830910538F421912093F10061505B
:1033B00071090196F3CF21E0089709F020E0809190
:1033C000E8008E778093E800CECF2111CFCF0AC0DE
:1033D0008091A501882361F0853061F08091E8003B
:1033E00083FD0AC08091E80082FFF2CF80E008955B
:1033F00082E0089583E0089581E008950F931F937C
:10340000CF93DF938B01EA019091A501943079F578
:103410008F708093E9008FEF9091E800815095FDC7
:1034200006C095ED9A95F1F700008111F5CF8091D6
:10343000E80085FF1CC00E942716882361F0809158
:10344000E8008E778093E80012C0F80181918F0127
:103450008093F1002197209791F38091E80085FDFA
:10346000F4CF8091E8008E778093E800E4CFDF917D
:10347000CF911F910F910895CF93DF93EC0148E016
:1034800050E0BC0181E00E94FE1988E0FE01ABE93A
:10349000B1E001900D928A95E1F7DF91CF91089507
:1034A00081E08093E00080E28093D8001092C90010
:1034B0008FE19EE40197F1F700C0000087E090EBF8
:1034C000DC018093000290930102A0930202B0936A
:1034D00003029CE088E10FB6F894A8958093600001
:1034E0000FBE90936000FFCF78941F920F920FB69B
:1034F0000F9211248F939F93AF93BF938091E1011B
:103500009091E201A091E301B091E4010196A11D27
:10351000B11D8093E1019093E201A093E301B09388
:10352000E401BF91AF919F918F910F900FBE0F90CB
:103530001F9018952FB7F8946091E1017091E20106
:103540008091E3019091E4012FBF08952FB7F89483
:103550008091E1019091E201A091E301B091E40139
:103560002FBF08951F920F920FB60F9211248F93C1
:103570009F93AF93BF938091E001811113C080911D
:10358000E1019091E201A091E301B091E401419643
:10359000A11DB11D8093E1019093E201A093E3018D
:1035A000B093E401BF91AF919F918F910F900FBEA7
:1035B0000F901F901895E1EDF1E09281891301C001
:1035C0001282319691E0E73DF907B9F70895A3ED2E
:1035D000B1E0EFEF90E02D91821789F0EF3F19F401
:1035E000211101C0E92F9F5F9630A9F7EF3F39F015
:1035F0000E2E000CFF0BEF52FE4F828308950895AC
:10360000E091DE01F091DF01309729F00190F08127
:10361000E02D0995089580E0089587E290E00E94EA
:1036200010200895CF93C82F811102C06FEF01C001
:1036300065E284E290E00E941020C11102C06FEFA9
:1036400001C061E085E290E00E941020C11102C03B
:103650006FEF01C064E186E290E00E941020CF91FC
:10366000089584E290E00E94F21F853281F485E2A1
:1036700090E00E94F21F813051F486E290E00E94B7
:10368000F21F91E0843109F090E0892F01C080E0C1
:10369000817008950F931F93CF93DF93C42F122F40
:1036A000FC0185818823B1F04093DD010E94A61AB8
:1036B0009093DC018093DB0180E28C0F883008F06E
:1036C00074C0C77081E001C0880FCA95EAF70E94F4
:1036D000241E6BC08091DD01481349C02091DB019D
:1036E0003091DC014FB7F8948091E1019091E201B3
:1036F000A091E301B091E4014FBF821B930B883C82
:103700009105A8F5D0E2D10FC117E9F080E28C0F46
:10371000883040F4C77081E001C0880FCA95EAF78D
:103720000E941D1ED83080F581E0912F977001C056
:10373000880F9A95EAF70E94241E093359F560E52F
:1037400070E089E32AC0093319F460E570E002C033
:1037500060E070E0802F0E940F1FD83030F5212FDD
:10376000277081E001C0880F2A95EAF70AC080E23D
:103770008C0F8830D0F4C77081E001C0880FCA95E3
:10378000EAF70E941D1E11C0093351F460E570E094
:1037900089E309C060E070E0802F0E940F1FDFCF37
:1037A00060E070E0802F0E940F1FDF91CF911F918A
:1037B0000F910895CF93DF93C8E5D2E060E0CE018A
:1037C0000E9410202196C11584E0D807B9F7DF9137
:1037D000CF9108951F93CF93DF93962F8430E8F411
:1037E0006530D8F44E30C8F4632F122FC42FD0E0C8
:1037F000CC0FDD1F2CE1929FC00DD11D11249CE840
:10380000899FC00DD11D1124CE0188960E941020E1
:10381000612FCE0189960E941020DF91CF911F91D8
:103820000895A0E0B0E0E7E1FCE10C945920A12C60
:10383000E12CF12CB12C00E010E0C0E0D0E06701F9
:10384000C00ED11EFE01EE0FFF1FEC0DFD1DE85254
:10385000FD4F259134914C2F6B2D8A2D0E94EA1B30
:103860002196CE30D10571F7045E1F4FB39485E0E9
:10387000B812E3CF8CE8E80EF11CA39484E0A81200
:10388000D9CFCDB7DEB7EAE00C94752080E00E9476
:10389000121B60E070E0CB010E940D1B0E94111C06
:1038A0000E94DA1B81E00E94121B08950F931F9360
:1038B000CF93DF93843008F56530F8F44E30E8F4A8
:1038C000C42FD0E0CC0FDD1F2CE1629FC00DD11DB5
:1038D00011243CE8839FC00DD11D1124CE01889690
:1038E0000E94F21F90E0182F0027CE0189960E94B7
:1038F000F21F9801282BC90102C080E090E0DF91FF
:10390000CF911F910F9108958B3109F473C058F531
:103910008B3009F497C078F4863009F446C020F45F
:10392000853009F44CC092C0873009F455C0883006
:1039300009F488C08BC0803109F46FC068F48E3000
:1039400009F084C08091DA0182FB222720F991E0FE
:10395000922790FB82F957C0863109F473C08931F0
:1039600009F470C073C08A32E9F060F4873209F458
:103970006BC028F48E3108F469C08D5159C089326A
:10398000F1F064C0833450F48A3308F050C08533BA
:1039900009F45AC0883309F455C058C0833409F477
:1039A00053C054C00E94C80E4DC08091DA01817F7F
:1039B0008E7F8093DA0181E08093D90108950E947F
:1039C0000F1E2FEF84E39CE0215080409040E1F7F0
:1039D00000C000000E94501A8091DA01982F909543
:1039E000917090FB80F98093DA0191112BC0897F4F
:1039F000877F10C08091DA0181FB222720F991E0B6
:103A0000922790FB81F98093DA019923D9F0809174
:103A1000DA0181608093DA0115C08091DA0183FBBD
:103A2000222720F991E0922790FB83F9ECCF89536C
:103A300091E001C0990F8A95EAF7892F0E94E91D4C
:103A40000E940F1E81E0089581E0F8CF80E0089584
:103A5000CF92DF92FF920F931F93CF93DF936C016E
:103A60000091B90180919401082BC3E0D0E010E0EF
:103A7000C8010C2E02C0959587950A94E2F780FD47
:103A800004C02197A8F7F12C09C0FC2EB6018C2F99
:103A90000E949E0D0E94AC0D019799F38F2DDF912E
:103AA000CF911F910F91FF90DF90CF900895CF930A
:103AB000DF93EC010E94281DBE010E949E0D0E9412
:103AC000AC0DDF91CF910895292F953078F58E3088
:103AD00068F590E03EE0239F800D911D1124682F32
:103AE000677023E0969587952A95E1F7FC01EE0F24
:103AF000FF1FE80FF91FEB51FE4F40E050E080E060
:103B0000219130E0062E02C0369527950A94E2F7FF
:103B100021703327042E01C0220F0A94EAF7822B6A
:103B20004F5F5F4F4330510559F7089580E0089586
:103B3000292F953088F58E3078F590E03EE0239F70
:103B4000800D911D1124282F277051E001C0550FC1
:103B50002A95EAF723E0969587952A95E1F7FC01E7
:103B6000EE0FFF1FE80FF91FEB51FE4F20E030E092
:103B700070E04081CB01022E02C0969587950A9491
:103B8000E2F78170819584278523842781932F5FB5
:103B90003F4F2330310569F708958093B9010895A7
:103BA00021E030E001C0220F8A95EAF7209580914C
:103BB000B90182230E94CD1D089521E030E001C0AB
:103BC000220F8A95EAF78091B901822B0E94CD1DC0
:103BD0000895809394010895FC0124812223D9F053
:103BE000808191810E94571D92959F70963079F047
:103BF00010F4925001C09A50923068F4803F69F0FE
:103C000018F4883E40F409C0843F29F406C0883E79
:103C100020F0813F11F080E0089581E00895109236
:103C2000930186E0E3EDF1E0DF011D928A95E9F76B
:103C300010928A010E943C0F0895882321F00E946F
:103C4000350F0E943C0F0895882339F0909193011D
:103C5000892B809393010E943C0F08958823E9F1FA
:103C6000823859F40E94001B81FF37C089E30E940B
:103C7000E71A0E943C0F89E31EC0833859F40E9462
:103C8000001B80FF2AC083E50E94E71A0E943C0FB8
:103C900083E511C0843859F40E94001B82FF1DC0C7
:103CA00087E40E94E71A0E943C0F87E404C09CEF5F
:103CB000980F913A18F40E94DB1A0DC090E2980F09
:103CC000983058F4877091E001C0990F8A95EAF70F
:103CD000892F0E94350F0E943C0F0895CF938823AF
:103CE00009F49BC0C82F8238A1F40E94001B81FDFB
:103CF00094C089E30E94E71A0E943C0F2FEF87EEE1
:103D000093E0215080409040E1F700C0000089E33B
:103D10002BC08338A1F40E94001B80FD7EC083E588
:103D20000E94E71A0E943C0F2FEF81EE94E0215091
:103D300080409040E1F700C0000083E515C0843862
:103D4000B1F40E94001B82FD68C087E40E94E71A5C
:103D50000E943C0F2FEF81EE94E021508040904074
:103D6000E1F700C0000087E40E94DB1A3EC08CEF40
:103D70008C0F813A50F58091D901882319F0813058
:103D800049F01DC0809193018232A1F58C2F0E94D1
:103D9000841C18C0809193018232C1F3C43149F070
:103DA00018F4CB3049F024C0C93219F0C83321F0DF
:103DB0001FC01092D9011CC081E0817003C0109215
:103DC000D90118C0811129C015C080E28C0F88303C
:103DD00020F5C77081E090E001C0880FCA95EAF72E
:103DE00090919301892B809393010E943C0F15C001
:103DF00080E0E3CFE3EDF1E08191C81741F021E0ED
:103E0000E93DF207C9F78C2F0E94E71AEECF8C2FFD
:103E10000E94DB1A0E943C0FF6CFCF9108951F93AA
:103E2000CF93DF93182FEB010E946E1E209741F075
:103E30008FE99FE00197F1F700C000002197F6CFCE
:103E4000812F0E942E1EDF91CF911F910895A6E031
:103E5000B0E0EDE2FFE10C94602049835A83498190
:103E60005A81992361F0222351F0CA010E94281D32
:103E7000182F682F89819A810E94981D04C0CA0159
